:100000000C9462000C94F71A0C94241B0C948A0034
:100010000C948A000C948A000C948A000C948A0038
:100020000C948A000C948A000C948A000C948A0028
:100030000C948A000C94C2060C948A000C948A00DA
:100040000C94511B0C948A000C94A41E0C94DF1E7B
:100050000C948A000C948A000C948A000C948A00F8
:100060000C9446050C948A00000000002400270030
:100070002A0000000000250028002B0000000000DE
:1000800023002600290004040404040404040202DA
:100090000202020203030303030301020408102007
:1000A0004080010204081020010204081020000012
:1000B0000007000201000003040600000000000029
:1000C0000000872011241FBECFEFD8E0DEBFCDBFD8
:1000D00012E0A0E0B1E0E4E1F3E402C005900D928B
:1000E000A43CB107D9F714E0A4ECB2E001C01D9222
:1000F000AE3AB107E1F710E0C4ECD0E004C02297BB
:10010000FE010E948421C23CD107C9F70E94CC2085
:100110000C9488210C940000FB01DC0102C00190CA
:100120000D9241505040D8F708958091C40281301B
:1001300019F482E08093C4028091C402833019F4E0
:1001400084E08093C4020895E3E0F0E089E08093C6
:100150005700849190E08670863009F491E0892FF1
:1001600008951F93182F0E94A400882379F09FB749
:1001700081E08093F403F894A89588E1809360006F
:1001800010936000112309F0A8959FBF1F91089557
:10019000382F20E08091F5039091F6038227932772
:1001A00040E061E270E19C01220F331F97FF04C021
:1001B000C9018627972701C0C9014F5F483099F7C9
:1001C0009093F6038093F50308958436910520F407
:1001D000BC0180E090E025C08E3B910550F48A552B
:1001E0009040BC0180E090E02AE030E040E050E048
:1001F00016C0823D910550F4845B9040BC0180E0C4
:1002000090E024E630E040E050E009C08D5C904092
:10021000BC0180E090E028E532E040E050E00E9440
:10022000DB2024E630E040E050E00E94DB2008952F
:1002300090E08C599F4F0E94E5000895DC0198964C
:10024000EC91F0E0E770F070E455FD4F8081089587
:10025000FC0120A530E0C9018170907001962770E3
:10026000307035952795820F931F880F880F08955A
:100270008F929F92AF92BF92CF92DF92EF92FF92B6
:100280000F931F938C010E941E01D80197962C9109
:1002900030E043E150E0249FF001259FF00D349FB2
:1002A000F00D1124EC50FE4F80809180A280B3802D
:1002B00090E00F96AA2797FDA095BA2FBC01CD011B
:1002C00020E43FE14DE750E00E94DB20A5019401CE
:1002D0000E940E2169017A0180ED97E0A0E0B0E074
:1002E000C80ED91EEA1EFB1ED80198968C91887103
:1002F00081F060E07EEE8AEB9BE0A50194010E9414
:100300000E2128513C4F4F4F5F4FC20ED31EE41EAB
:10031000F51E87EE93E0A0E0B0E0C80ED91EEA1EFD
:10032000FB1EC701B60128EE33E040E050E00E941A
:100330000E21CA01B90128EE33E040E050E00E94EE
:10034000DB201F910F91FF90EF90DF90CF90BF9037
:10035000AF909F908F9008951F93182FDB01FA01A3
:10036000482F469530E0848190E083709070982FFC
:1003700088272081820F911D11969C938E938481F2
:1003800090E08C70907076E0880F991F7A95E1F775
:100390002181820F911D13969C938E9312978481D5
:1003A00090E08073907064E0880F991F6A95E1F780
:1003B0002281820F911D15969C938E9314978481B0
:1003C00090E0807C9070880F991F880F991F23817F
:1003D000820F911D17969C938E93169735961896BB
:1003E0003F5F431708F0BFCF10FF50C08081829558
:1003F00086958695837090E02DE431E0AC01429FB4
:10040000C001439F900D529F900D11240C961196A0
:100410009C938E93808190E044E0969587954A95D1
:10042000E1F783709070AC01429FC001439F900D33
:10043000529F900D11240C9613969C938E931297B5
:10044000808190E0969587959695879583709070BA
:10045000AC01429FC001439F900D529F900D11240B
:100460000C9615969C938E931497808190E08370E0
:100470009070AC01429FC001439F900D529F900D20
:1004800011240C9617969C938E9316971F9108959E
:1004900023E08032920718F420E030E026C023E009
:1004A000883E920748F49C012F51334054E0369522
:1004B00027955A95E1F719C027E0803D920720F46F
:1004C0009C012C5D334011C028E08839920718F058
:1004D0002FEF33E00AC09C01285C374044E036959A
:1004E00027954A95E1F72D503C4FC90108958C306E
:1004F000910548F49C0174E0220F331F7A95E1F7CF
:10050000285D3C4F17C023E0843F920720F49C01F4
:1005100024523C4F0FC024E08030920718F020E9AD
:1005200038E008C09C012657334F64E0220F331F88
:100530006A95E1F7C90108959C01369527952575BF
:100540003575821B930B9C0136952795369527951B
:100550002373337383739373280F391FC901E4E046
:1005600096958795EA95E1F7820F931F8F709F709C
:1005700021E031E0AC01429FC001439F900D529FAA
:10058000900D1124892F0895882339F02D980000AB
:100590002B9A00002D9A000008952D9800002B98AA
:1005A00000002D9A000008952D9A000083B12D9827
:1005B000000090E0B4E096958795BA95E1F78170D8
:1005C00008950F931F93082F5C9A2D985C9810E064
:1005D000802F80780E94C402000F1F5F1830C1F77F
:1005E0002D981F910F9108958F770E94E102089531
:1005F0000F931F93082F10E0802F80780E94C40271
:10060000000F1F5F1830C1F72D981F910F910895AB
:100610000F931F932D9880E000E0182F110F0E9478
:10062000D402810F0F5F0830C1F71F910F91089519
:100630000E94F4020E9408035C9A08951F93162FEB
:1006400080680E94E102812F0E94F8025C9A1F914B
:1006500008951F931091E9021827E0EEF2E0E80FE9
:10066000F11D89E767850E941E038DE3612F0E94BB
:100670001E0382E4612F0E941E031F91089586E2EB
:100680000E94180308950F931F938BE20E94180392
:10069000082F8CE20E941803282F30E096E0369550
:1006A00027959A95E1F710E0000F111F000F111F19
:1006B000202B312BC9011F910F9108950F931F9388
:1006C0008C018CE1F80164810E941E038DE1F80128
:1006D00065810E941E038EE1F80166810E941E035F
:1006E00080E2F80167810E941E0381E2F8016085C3
:1006F0000E941E0382E2F80161850E941E0383E2CC
:10070000F80162850E941E0384E2F80163850E945D
:100710001E0385E2F80164850E941E038AE2F80147
:1007200065850E941E038EE6F80166850E941E0301
:100730008FE6F80167850E941E0380E7F801608953
:100740000E941E0381E7F80161890E941E0382E76F
:10075000F80162890E941E031F910F910895EF9284
:10076000FF920F931F93CF93DF937B018C01603037
:1007700028E372072CE982072CE1920728F520E88C
:1007800036E948E950E00E940E21E9016897B90175
:1007900080E090E020E839E647E65FEF0E94DB204A
:1007A0006E0D7F1D801F911F32E0660F771F881F1F
:1007B000991F3A95D1F721E732E040E050E00E94DE
:1007C0000E21890180E421C020E03DE241E351E0B7
:1007D0000E940E21E9016897B90180E090E020E0D5
:1007E00033ED4EEC5EEF0E94DB206E0D7F1D801F0F
:1007F000911F660F771F881F991F21E732E040E0A5
:1008000050E00E940E21890180E69E012F71622F27
:10081000680F85E70E941E0386E7612F0E941E0372
:1008200087E7602F0E941E03CDB7DEB7E6E00C9489
:1008300073219F92AF92BF92CF92DF920F93DF937B
:10084000CF9300D000D0CDB7DEB7982E83E00E94C2
:1008500018038093090384E00E94180380930A031D
:1008600086E060E00E941E0387E061E00E941E03B4
:1008700089E06FE70E941E038AE065E00E941E0384
:100880008BE062E10E941E038CE065E10E941E0382
:100890008DE06DEF0E941E038EE060E00E941E035B
:1008A000992019F083E592E008C08091070323E1C5
:1008B000829FC00111248C509E4F0E945E0380E3F2
:1008C0006CE80E941E0382E36FE00E941E0383E334
:1008D00062E40E941E0384E36AE00E941E0385E333
:1008E0006AE20E941E0386E36DE20E941E0387E314
:1008F00064ED0E941E0388E360E00E941E0389E30A
:1009000060E00E941E03992049F065E8A62E61EC84
:10091000B62E61ECC62E6EEDD62E08C0A090E90270
:10092000B090EA02C090EB02D090EC020AE38D2D69
:100930009927AA27BB2789839A83AB83BC83802FFF
:1009400069810E941E03802F8B5F69810E941E03B4
:10095000DC2CCB2CBA2CAA240F5F0E3341F783E496
:100960006FEF0E941E0384E46FEF0E941E0385E474
:100970006FEF0E941E0386E46FEF0E941E03992012
:1009800019F08DE666E003C08DE66091ED020E94ED
:100990001E0389E760E00E941E038AE76091EE0271
:1009A0000E941E0383E760E00E941E0384E760E06C
:1009B0000E941E03992029F060EC72E98DEE99E106
:1009C00008C06091E5027091E6028091E702909183
:1009D000E8020E94AF030F900F900F900F90CF91FD
:1009E000DF910F91DF90CF90BF90AF909F900895CF
:1009F00087E061E00E941E038EE764E20E941E030E
:100A000088E063E00E941E0388E060E00E941E030D
:100A100087E065E00E941E0385E062E00E941E03FD
:100A200083E00E9418038093090384E00E94180366
:100A300080930A03089590E0411191E0880F982B6C
:100A40009093BA00660F6093BD003093100320931B
:100A50000F030895882311F085EC01C085E8809389
:100A6000BC00089585ED8093BC008091BC0084FD9E
:100A7000FCCF089585EC8093BC000895ECEBF0E08A
:100A8000108285E480831092150308951F920F92BF
:100A90000FB60F9211242F933F934F935F936F9351
:100AA0007F938F939F93AF93BF93EF93FF93DF93C6
:100AB000CF930F92CDB7DEB78091B90090E0887FD9
:100AC00090708036910509F4EAC081369105CCF525
:100AD0008832910509F47CC089329105B4F48031E3
:100AE000910509F470C0813191053CF4009709F437
:100AF0000EC1089709F00DC166C08831910509F44F
:100B000067C0809709F005C177C08034910509F46A
:100B100090C08134910544F48033910509F46EC08E
:100B2000C89709F0F6C06CC08035910509F471C012
:100B30008835910509F483C08834910509F0E9C02E
:100B4000A5C08839910509F4DCC089399105ECF418
:100B50008837910509F4A3C0893791054CF488368C
:100B6000910509F49CC08037910509F0D2C097C067
:100B70008838910509F4C5C08039910509F492C0FF
:100B80008038910509F0C5C08DC0803B910509F4FE
:100B9000A5C0813B91054CF4803A910509F499C0B8
:100BA000883A910509F0B5C099C0803C910509F4D7
:100BB000AAC0883C910509F4A6C0883B910509F0BC
:100BC000A8C080E08CC0809111038093BB009BC0C3
:100BD000809114038150809314038F5F09F43FC008
:100BE000E0911203F091130381918093BB00F09385
:100BF0001303E093120387C082E049C083E047C03B
:100C000084E080931603809115038B7F80931503F6
:100C100062C08091BB00E0911203F09113038193B5
:100C2000F0931303E0931203809114038150809397
:100C3000140380911403823008F065C062C0809173
:100C4000BB00E0911203F09113038193F09313031F
:100C5000E0931203809114038150809314038091D8
:100C600015038B7F809315038091150380FF4FC080
:100C7000809115038E7F8093150380911503826008
:100C80008093150384EA8093BC0043C085E0809381
:100C90001603809115038B7F8093150338C0109243
:100CA000140331C0E0910F03F0911003309749F124
:100CB0009091BB00809114038F5F80931403815047
:100CC00011F060E001C062E09983CE0101960995C0
:100CD0001BC00E9432050E943A051BC081E0E091D2
:100CE0000F03F0911003309761F0882311F461E055
:100CF00001C063E0CE010196099599819093BB00F4
:100D000003C080E001C081E00E942A0502C00E9469
:100D100032050F90CF91DF91FF91EF91BF91AF918D
:100D20009F918F917F916F915F914F913F912F9103
:100D30000F900FBE0F901F90189525B190E0FC0109
:100D4000EE0FFF1FE80FF91FE458FC4F8081282B9E
:100D500025B988B19181892B88B98BB19281892B72
:100D60008BB9089585B19091AC03892385B988B179
:100D70009091AD03892388B98BB19091AE038923FB
:100D80008BB908951F920F920FB60F9211241F93E3
:100D90002F933F934F935F936F937F938F939F9383
:100DA000AF93BF93CF93DF93EF93FF9310914F03D4
:100DB00080918A02C0918802D0918902181708F0A8
:100DC0005BC08091AF039091B003909387008093B4
:100DD0008600E12FF0E0EE0FFF1FEA59FD4F808102
:100DE00091810E947702880F991F9093B00380939E
:100DF000AF038091AF039091B0039E01281B390B84
:100E0000C90130938902209388022091DB0230913E
:100E1000DC02220F331F8217930720F430938902DC
:100E20002093880280915103882339F48091D30262
:100E300080FF59C0183008F456C08FEF9FEF909391
:100E4000890080938800809184009091850080972C
:100E5000D0F30E94B20680915003882339F4809128
:100E60004F03882319F081500E949D0680914F0303
:100E70008F5F80934F033EC08091AF039091B0038A
:100E80009093870080938600D093B003C093AF0304
:100E900080915103882319F08FEF9FEF06C0809156
:100EA000AF039091B003885592409093890080934E
:100EB000880080E49CE99093890280938802809165
:100EC0008400909185008097D0F30E94B2068091B3
:100ED0005003882329F480918A0281500E949D0644
:100EE00010924F0307C08091AF039091B0038855D3
:100EF0009240A5CFFF91EF91DF91CF91BF91AF913C
:100F00009F918F917F916F915F914F913F912F9121
:100F10001F910F900FBE0F901F90189590E0880FB3
:100F2000991F880F991F8C30910518F42CE030E040
:100F300007C09C0183E0253F380710F024EF33E021
:100F4000C90108950F931F930091D4020033C0F498
:100F5000202F30E0C90180739070009719F04097FE
:100F600049F403C08091490307C080914E038295E4
:100F7000807F02C08091480389010F70107016C0F5
:100F80000F33E8F410E00F70107080914E038295DB
:100F9000807F0E948E07F801EE0FFF1FEA59FD4F78
:100FA000918380830F5F1F4F809148030E948E07BB
:100FB000000F111F0A591D4FF801918380831F9163
:100FC0000F9108951F9380915303909154038F5F65
:100FD0009F4F39F11091D402412F50E04F70507063
:100FE000BA016F5F7F4FA3E5B3E020E030E0241744
:100FF000350789F02617370711F4103360F4F89499
:101000008D919C911197F901EE0FFF1FEA59FD4F49
:101010009183808378942F5F3F4F12962031310562
:1010200031F71F9108951F93CF93DF93EC0170E088
:10103000CB018270907060FF1AC0892B31F08091D3
:10104000750388831092F30345C01091F30380EE7B
:1010500092E00E941E011817D8F5E12FF0E0EF543E
:10106000FC4F808188831F5F1093F30333C0892B6B
:10107000C1F098819093F2031092F303892F807E40
:10108000803651F480917503823010F188818F7120
:101090008093330383E01AC09E3FE1F410927503FE
:1010A00017C08091F2038F3FA9F42091F3032932F6
:1010B00078F4E22FF0E0E052FD4F88818083822FA8
:1010C0008F5F8093F303893229F481E08093750365
:1010D00080E001C081E0DF91CF911F910895EF92F0
:1010E000FF920F931F93CF93DF9380E260E040E085
:1010F00023E138E00E941B051092750392E0E92E6F
:1011000085E0F82E04E080917503813039F480E0A9
:101110000E941904E09275035E98F5CF1091750353
:10112000133061F45D98809133030E94290310937A
:10113000C4020E94F80400937503E5CF8091750303
:10114000843009F78091C4028430E9F68FE70E9469
:10115000F402C0E0D0E007C00E940803FE01EF5493
:10116000FC4F8083219680EE92E00E941E0190E069
:10117000C817D9078CF3F09275035D9AC4CFA0E02D
:10118000B0E0E5ECF8E00C945321EC010E94A71BC1
:101190005B016C017E0100E010E011C0209779F046
:1011A0000E94A71B6A197B098C099D09E616F706A0
:1011B0000807190720F40E943E0581E008C08091CD
:1011C000150382FDEBCF8091160310921603CDB765
:1011D000DEB7EAE00C946F21A0E0B0E0E2EFF8E0C7
:1011E0000C945521182F7B01042FC22FD0E024E04E
:1011F000C22ED12CCC22DD22C2FF03C080E090E0C1
:1012000004C080918602909187020E94BF08282F17
:101210008823B9F51092160300931403F092130378
:10122000E0921203110F11601093110390911503B6
:10123000C1FD02C084E001C085E0892B80931503C5
:101240008091150381FF0BC0809115038D7F8093E2
:101250001503809111038093BB0085EC01C085EEDE
:101260008093BC00C0FF0DC0C114D10419F080E010
:1012700090E004C080918602909187020E94BF088E
:10128000282F822FCDB7DEB7E8E00C947121A0E0C3
:10129000B0E0EDE4F9E00C945521182F7B01042F08
:1012A000C22FD0E034E0C32ED12CCC22DD2222FF8D
:1012B00003C080E090E004C0809186029091870294
:1012C0000E94BF08282F8823B1F5109216030093BF
:1012D0001403F0921303E0921203110F1093110301
:1012E00090911503C1FD02C084E001C085E0892B07
:1012F000809315038091150381FF0BC08091150326
:101300008D7F80931503809111038093BB0085EC42
:1013100001C085EE8093BC00C0FF0DC0C114D10494
:1013200019F080E090E004C08091860290918702DD
:101330000E94BF08282F822FCDB7DEB7E8E00C94BB
:1013400071218091C402813011F081E008950E94E2
:10135000A71B20910B0330910C0340910D0350917A
:101360000E03621B730B840B950B615A7648814008
:10137000904010F480E0089582E00895FF920F936A
:101380001F93CF93DF93182F092FF62E8EE30E9421
:101390001E03212F302FC901EC0110E005C08FE79B
:1013A00069910E941E031F5F1F15C8F385E064E06A
:1013B0000E941E0383E00E9418038093090384E0C7
:1013C0000E94180380930A030E94A71B60930B03DB
:1013D00070930C0380930D0390930E0387E069E0F4
:1013E0000E941E0381E08093C402CDB7DEB7E5E022
:1013F0000C9474210E94BE098091C4028130D9F4FA
:101400000E94A71B20910B0330910C0340910D0308
:1014100050910E03621B730B840B950B605A764838
:101420008140904040F4E8CF8CE894E060E071E0C7
:101430000E948F1E08958091C4028130A9F30895FF
:10144000A1E0B0E0E6E2FAE00C945B218091750344
:101450008230B9F480E2BE016F5F7F4F41E021E04E
:101460000E94EC08882379F08FEF809375030E9427
:10147000991B60937603709377038093780390931E
:1014800079038FEF01C089812196E2E00C947721E6
:10149000A1E0B0E0EEE4FAE00C945B2180917503EA
:1014A0008230D9F480913303805A898380E2BE016F
:1014B0006F5F7F4F41E021E00E944709882369F078
:1014C0008FEF809375030E94991B6093760370934E
:1014D000770380937803909379032196E2E00C944C
:1014E0007721AAE2B0E0E7E7FAE00C9459218FEF08
:1014F0008983DE011296E0EEF2E089E201900D921E
:101500008150E1F780E28E010F5F1F4FB8014AE280
:1015100021E00E944709882351F480E2B80141E0AC
:1015200021E00E94EC08882311F482E001C08FEFD3
:101530008093750380917503823051F00E94991B4E
:101540006093760370937703809378039093790385
:10155000AA96E4E00C947521A2E0B0E0E2EBFAE098
:101560000C9457210E94A71B9B01AC01809117038B
:1015700090911803A0911903B0911A0379018A017F
:10158000E81AF90A0A0B1B0BD801C70181519742CF
:10159000A040B04008F444C080911B038F5F80934B
:1015A0001B03815080FD02C000E001C007E02093D2
:1015B0001703309318034093190350931A038CE8D0
:1015C00094E063E00E9447208CE894E061E00E9490
:1015D000472077E0F72EF00E802F90E0880F991FBC
:1015E0009C012A593D4F3A832983F9016081718119
:1015F000672F772763707070880F991F682B792B7E
:101600008CE894E00E944720E981FA816081718131
:1016100070708CE894E00E9447200F5F0F15E1F690
:101620002296E6E00C9473211F93182F8CE894E027
:10163000612F0E944720812F0E94C8001F910895AA
:10164000A0E0B0E0E6E2FBE00C945521082F0E94F8
:10165000A71B9B01AC018091170390911803A091E7
:101660001903B0911A0369017A01C81AD90AEA0A62
:10167000FB0AD701C60181519742A040B04008F44F
:1016800043C02093170330931803409319035093DA
:101690001A031092F6031092F50388EA0E94140BC5
:1016A000002311F481E001C081E80E94140B80E165
:1016B0000E94140BC0E0D0E0FE01EE0FFF1FEA59BC
:1016C000FD4F808191810E9477028C01E3E0000F41
:1016D000111FEA95E1F7812F0E94140B802F0E94C1
:1016E000140B2196C031D10539F76091F6038CE8CF
:1016F00094E00E9447206091F5037091F6037070AA
:101700008CE894E00E944720CDB7DEB7E8E00C9467
:101710007121A0E0B0E0EFE8FBE00C945521182F18
:10172000062F0E94A71B9B01AC018091170390918B
:101730001803A0911903B0911A0369017A01C81A1C
:10174000D90AEA0AFB0AD701C60181519742A04093
:10175000B04008F4D6C12093170330931803409388
:10176000190350931A038091660290916702880FC3
:10177000991F80931C03977080911D03887F892B8C
:1017800080931D032091680230916902220F331F5C
:10179000922F990F990F990F8770892B80931D03B2
:1017A000422F42954695477080911E03807C932F6F
:1017B0009770990F990F990F842B892B80931E0393
:1017C00020916A0230916B02220F331F922F929563
:1017D000990F990F907C8F73892B80931E03932F01
:1017E0009295990F990F907C822F86958695892BDB
:1017F00080931F03932F9695969591708091200367
:101800008E7F892B8093200320916C0230916D0292
:10181000220F331F922F990F8170892B8093200301
:10182000422F441F4427441F80912103807F932F20
:101830009770990F842B892B8093210320916E023E
:1018400030916F02220F331F922F9295907F8F70ED
:10185000892B80932103422F42954F708091220360
:101860008078932F97709295907F842B892B80930B
:1018700022032091700230917102220F331F8F7763
:1018800080932203932F979599279795822F86957A
:10189000892B80932303932F969593708091240333
:1018A0008C7F892B809324034091720250917302A4
:1018B000440F551F942F990F990F8370892B809394
:1018C0002403942F929596959695937020912503D5
:1018D000207E852F8770880F880F292B282B209337
:1018E00025038091740290917502880F991F382FFB
:1018F0003295330F307E2F71232B20932503292F10
:101900002295220F207E869586958695822B809340
:1019100026038091760290917702880F991F809319
:101920002703977080912803887F892B8093280351
:101930002091780230917902220F331F922F990F54
:10194000990F990F8770892B80932803422F429516
:101950004695477080912903807C932F9770990F4B
:10196000990F990F842B892B8093290320917A0258
:1019700030917B02220F331F922F9295990F990F6E
:10198000907C8F73892B80932903932F9295990FC5
:10199000990F907C822F86958695892B80932A03B8
:1019A000932F96959695917080912B038E7F892B1E
:1019B00080932B0320917C0230917D02220F331FF4
:1019C000922F990F8170892B80932B03422F441FF4
:1019D0004427441F80912C03807F932F9770990F89
:1019E000842B892B80932C0320917E0230917F02DF
:1019F000220F331F922F9295907F8F70892B8093A7
:101A00002C03422F42954F7080912D038078932FA5
:101A100097709295907F842B892B80932D03209132
:101A2000800230918102220F331F8F7780932D0324
:101A3000932F979599279795822F8695892B809339
:101A40002E03932F9695937080912F038C7F892B73
:101A500080932F034091820250918302440F551FBF
:101A6000942F990F990F8370892B80932F03942FB4
:101A7000929596959695937020913003207E852FB0
:101A80008770880F880F292B282B20933003809193
:101A9000840290918502880F991F382F3295330F59
:101AA000307E2F71232B20933003292F2295220F74
:101AB000207E869586958695822B8093310311230F
:101AC00011F490E001C098E0002311F480E001C01F
:101AD00084E0892B809332038CE894E06FE00E94CD
:101AE0004720CCE1D3E08CE894E069910E94472044
:101AF00083E0C333D807B9F78CE894E060E00E9434
:101B00004720CDB7DEB7E8E00C9471211F93182F62
:101B10008091CB028B3221F48FE0612F0E94A21CB6
:101B20008091C802873259F4112321F08091B000CE
:101B3000806103C08091B0008F7E8093B0001F91C0
:101B4000089580914C0390914D039F770E949C02D1
:101B5000982F80934E038F3029F480914803869507
:101B6000805804C089E0989FC001112480934903E4
:101B7000F8940E94A20778948091C8028132C9F437
:101B800090914903892F81508E3F60F08091B00081
:101B90008F7D8093B00060E0911161E083E00E944E
:101BA000A21C08959093B4008091B000806280934D
:101BB000B00008951F93182F811111E082E1612F69
:101BC0000E94A21C83E1612F0E94A21C10921403A8
:101BD000109215038091B9008C6F8093B90080E258
:101BE0008093B80085E48093BC001F910895CF9343
:101BF000DF938CE894E00E94D41F892BF9F0809148
:101C0000F003C82FD0E09E012F5F3F4F2F7130703F
:101C10008091EF0390E02817390781F08CE894E079
:101C20000E940E20C153DC4F88838091F00390E026
:101C300001968F7190708093F003DBCFDF91CF918D
:101C40000895EF92FF921F93CF93DF9380EE92E07F
:101C50000E942801482F80938A025091D402252F98
:101C600030E02F70307090E02817390719F44F5F7B
:101C700040938A0250535F3058F440918A02842F77
:101C800090E001972817390719F44F5F40938A02B3
:101C900080918A02813118F080E180938A02ECE71A
:101CA000F3E0108211821282339623E0E439F207C6
:101CB000C1F78FEF8093AC038093AD038093AE03A5
:101CC00086ECE82E82E0F82EA4E9B2E0E7016FEF9F
:101CD0005FEF4FEF88818031F0F490E03C91FC01A0
:101CE000EE0FFF1FE80FF91FE458FC4F8081832B94
:101CF000808311962C9111978181822B818312967A
:101D00009C9112978281892B828330954323209561
:101D10005223909569232196139682E0CE3CD807F2
:101D2000C9F66093AE035093AD034093AC03CCE887
:101D3000D2E010E0F7018081823238F08632B0F0D4
:101D4000863219F4888160E00FC0163021F480914A
:101D5000C1008F7E05C0173029F48091C100877FB4
:101D60008093C100888161E00E94361C1F5F089447
:101D7000E11CF11C21961830E9F68091C6028032F0
:101D800031F489E061E00E94A21C82E801C082E097
:101D90008093800081E08093500380935103809171
:101DA000C802813211F08732D9F483E061E00E94E9
:101DB000361C83E060E00E94A21C8091C802813240
:101DC00031F481E08093B0008093B10009C082E0DB
:101DD0008093B00085E08093B1008EE38093B300E0
:101DE0008AE1809381008FEF9FEF90938900809329
:101DF000880080ED97E0909387008093860080E4D0
:101E00009CE990938902809388029093B003809319
:101E1000AF0310924F0380916F00816080936F0039
:101E20008091D30283FF0DC080915303909154039E
:101E30008F5F9F4F31F00E94E20710925103109282
:101E40005003DF91CF911F91FF90EF9008958CE0A8
:101E500060E00E94361C8BE061E00E94361C8DE041
:101E600061E00E94361C82E060E00E94361C84E043
:101E700061E00E94361C089583E00E94180380935D
:101E8000090384E00E94180380930A0387E061E05D
:101E90000E941E036AE070E080E090E00E94CD1B8B
:101EA0000E94F804000008950F931F93082F17C095
:101EB0005E9A64E670E080E090E00E94CD1B5E9840
:101EC00064E670E080E090E00E94CD1B1F5F101779
:101ED00078F36CE271E080E090E00E94CD1B10E0AE
:101EE000F6CF482F392F25E00DC0F999FECF1FBA44
:101EF000842F932F92BD81BD60BD0FB6F894FA9ADE
:101F0000F99A0FBE215059F0F999FECF842F932FE3
:101F100092BD81BDF89A80B5681739F7089582E0BF
:101F20000E94540F0895A0E0B0E0E9E9FFE00C94AE
:101F30004D21482E562EEE24FF24C0E0D0E0CC24C4
:101F4000DD248824992404C055245394CC24DD2412
:101F5000442051F465ECE62E62E0F62EC0E0D0E0BD
:101F60005BE1852E912C19C021E0421651F440EE20
:101F7000E42E42E0F42ECDE1D0E039E2832E912C24
:101F80000CC032E0431649F423E5E22E23E0F22EA2
:101F9000C8E4D0E090E2892E912C3E016C0C7D1CAF
:101FA0001092F6031092F503E3011BC0552059F47B
:101FB000F999FECFD2BDC1BDF89A80B5F701E00F07
:101FC000F11F808307C0F701E00FF11FCE01608190
:101FD0000E94710F0E0D1F1DF80180810E94C80024
:101FE00021969E012619022F10E008151905F0F21E
:101FF000CE015520D9F4F999FECFD2BDC1BDF89AD2
:1020000020B5F999FECF2196D2BDC1BD2197F89A8E
:1020100080B590E0B22EAA248A299B292091F5034D
:102020003091F6032817390759F48ECF2196609125
:10203000F6030E94710FCE016091F5030E94710FAB
:1020400080E091E0C80ED91E91E0C91693E0D90650
:1020500008F47ECF852DCDB7DEB7E0E10C94692181
:1020600082E060E00E94930F882331F48FEF9FEFAE
:102070009093540380935303089582E061E00E949B
:10208000930F089595E09093C50290E29093C60255
:1020900092E29093C70291E29093C80293E29093E8
:1020A000C9029BE29093CB0294E29093CC0295E21A
:1020B0009093CD0292E09093D3029FEF9093D4023D
:1020C0002AE02093DD021092DE021092DF021092CD
:1020D000D5021092D6021092D7021092D8029EE139
:1020E0009093D9022093DA0228EB3BE03093DC0294
:1020F0002093DB02882361F080E061E00E94930F6F
:102100008FEF9FEF90935403809353030E943D10F1
:102110000895A3E6B0E0EFE8F0E10C944B215B01F9
:102120006C010E94991B1B012C0181E00E94190483
:1021300083E08093C4020E943C0F8CE894E06CE042
:1021400071E00E948F1E3E010894611C711C2FE3F8
:1021500030E02C0F3D1F2B5F3F4FA4963FAF2EAFBB
:10216000A497EEC08CE894E06AE171E00E948F1EB3
:102170008FE70E94F4020E940803182F8983823699
:1021800001F500EE12E00E940803F80181938F012F
:10219000F3E009301F07B9F78091E002873309F0B7
:1021A000CAC08CE894E063E271E00E948F1E82E472
:1021B0008983CE01019661E00E94FA095D9A81E06F
:1021C000D5C0803719F0893631F506C020E52A835D
:1021D000AA24BB24650105C081E00E94421089E465
:1021E0008A838091F403882321F08091D302806850
:1021F00003C08091D3028F778093D302DE011396C0
:10220000E5ECF2E08BE101900D928150E1F7CE0117
:1022100002966CE18EC0843731F584E58FAF33E0F0
:1022200021963FAF219783E722968FAF229788E0D0
:1022300023968FAF23978FE024968FAF2497A49691
:10224000AEADBFADA497E6EDF1E08EE101900D9249
:102250008150E1F7CE01CF9663E20E94FA09AA24E9
:10226000BB24650168C0853791F405EC12E00E943B
:102270000803F80181938F01F2E0003E1F07B9F7D0
:1022800080E061E00E94930F25E5298350C08636E7
:1022900031F580915303909154038F5F9F4FD1F09C
:1022A00086E48E8F73E5E72E73E0F72E8E01015ED4
:1022B0001F4FF701819191917F010E947702F801F0
:1022C000908381830E5F1F4FF3E7EF16F3E0FF0665
:1022D00081F701C01E8FCE014E9661E22AC087367B
:1022E000D9F403E513E00E940803982E88240E9485
:1022F00008039401280F311DC9010E944802F8010A
:10230000819391938F01F3E003371F0761F727E46F
:1023100029830E943D100BC0873469F48FEF9FEF33
:1023200090935403809353030E943D101983C3017B
:1023300061E00E94FA0993E09093C4020E94F804BD
:10234000A114B104C104D10459F00E94991B62196F
:102350007309840995096A157B058C059D0528F488
:102360008091C402843061F7FDCE80E0CD59DF4F0B
:10237000E2E10C94672180E060E00E94930F8823E3
:1023800019F481E00E944210089581E061E00E940A
:10239000930F089581E060E00E94930F882311F469
:1023A00090E006C090E08091E002873309F491E06C
:1023B000892F0895EF92FF920F931F93CF93DF938E
:1023C000EB019C01442737FD4095542F60E271EAF0
:1023D00087E090E00E94302189011216130614F064
:1023E00001E010E0BE01882777FD8095982F20E25C
:1023F00031EA47E050E00E94DB209801442737FD96
:102400004095542F0E9430217901C0E0D0E009C0EE
:102410002B9AC8010E94F11B2B98C8010E94F11B46
:102420002196CE15DF05A4F3CDB7DEB7E6E00C9418
:1024300073211F93182F5D9A83E00E9418038093E5
:10244000090384E00E94180380930A0386E060E099
:102450000E941E0387E061E00E941E0389E06FE78F
:102460000E941E038AE065E00E941E038BE062E189
:102470000E941E038CE065E10E941E038DE06DEF5B
:102480000E941E038EE060E00E941E0380E76CE263
:102490000E941E0380E360E00E941E0389E760E063
:1024A0000E941E038AE765E00E941E0381E762E145
:1024B0000E941E0382E762E00E941E0383E760E041
:1024C0000E941E0384E760E00E941E036091D50213
:1024D0007091D6028091D7029091D8020E94AF03EA
:1024E0008DE667E00E941E036AE070E080E090E005
:1024F0000E94CD1B87E069E00E941E036AE070E045
:1025000080E090E00E94CD1B112369F010E007C02D
:1025100088EB91E061E070E00E94DA11A8951F5FFE
:102520001531B1F74BC088E891E061E070E00E949E
:10253000DA11A8958DE665E00E941E036AE070E05E
:1025400080E090E00E94CD1B88EB91E061E070E0BC
:102550000E94DA11A8958DE664E00E941E036AE0ED
:1025600070E080E090E00E94CD1B8DE591E061E09D
:1025700070E00E94DA11A8958DE662E00E941E03C9
:102580006AE070E080E090E00E94CD1B8FEA90E06E
:1025900061E070E00E94DA11A8958DE660E00E948B
:1025A0001E036AE070E080E090E00E94CD1B85E0B1
:1025B00091E062E070E00E94DA11A89587E061E0A6
:1025C0000E941E035D981F910895A6E1B0E0EBEE16
:1025D000F2E10C944D21A8958CE00E941803882309
:1025E00059F48CE894E06EE271E00E948F1E80E066
:1025F0000E9419040E943C0F0E94F70D0E94A71B25
:102600000E94200A90E0853009F491E08E010F5F6E
:102610001F4FBB24BA948091C402843019F09923CF
:1026200009F494C10E94A71B6B017C018091C40234
:102630008430F1F48FE70E94F40200E010E008C05B
:102640000E940803F801EF54FC4F80830F5F1F4F77
:1026500080EE92E00E941E0190E00817190784F3B3
:102660000E94430390934B0380934A035D9A29C0D1
:1026700080EE92E00E941E01482F4F5F80E2B80179
:1026800021E00E94EC08882371F0B09275030E944B
:10269000991B6093760370937703809378039093EC
:1026A000790390E0B8CF80EE92E00E941E01482F9F
:1026B00021EB33E0FE013296C901BF0150E00E94D8
:1026C0008C00C0923403D0923503E0923603F0922E
:1026D00037031092740380914C0390914D03880F3F
:1026E000991F816090934D0380934C035E9880E026
:1026F0000E94860D8091B103282F30E0C9018E73AE
:102700009070892B99F5F89480910803877066E69C
:1027100072E042EB53E00E94AC010E94A207789461
:102720008091B10390917B0380FF1BC0992309F036
:1027300045C0A3E5B3E020E030E0F901EE0FFF1F54
:10274000EA59FD4F808191818D939D932F5F3F4F7B
:102750002031310591F70E943D1081E080937B0389
:102760002DC0992359F110927B0328C0C9018873A9
:102770009070C89719F54091C603842F822787FF70
:102780001DC040584093C6038091CD028532B1F4FC
:1027900010E00AC01F5FE12FF0E0EF54FC4F8CE81F
:1027A00094E060810E944720212F30E08091B103A6
:1027B00090E0877090708217930764F7809173039D
:1027C000882319F481E080937303109252031092CE
:1027D00050031092510380910803887109F4ADC031
:1027E0004091C6038091B10390E0242F30E082270E
:1027F000932786FD6CC0407C80E448274093C60345
:102800009091EF038091F003981701F1A7ECB3E0EA
:1028100030E00FC03F5F892F90E0FC01E153FC4F97
:1028200020812D9301968F7190708093EF03383043
:1028300031F09091EF038091F003981759F7395CCC
:102840008091C603382B3093C60341C08091470363
:102850008093C7038091C702863211F482E105C0DC
:102860008091CA02863251F48EE00E94051D959532
:102870008795959587958093C80302C01092C803E9
:102880008091C902863211F483E105C08091CB02A8
:10289000863251F48FE00E94051D95958795959598
:1028A00087958093C90302C01092C90380914B039E
:1028B0008093CA0380914A038093CB0380914C0399
:1028C00090914D039F770E949C028093CC0386ECED
:1028D00093E069E00E94BE0902C00E94F70D0E94C9
:1028E000A1098823D1F306EC12E08CE8E82E82E0FF
:1028F000F82EF8018081E82FF0E0CF01807F907002
:10290000409791F4EF70F070EE0FFF1FEA59FD4F02
:102910008081918160E08F3F910511F008F061E0C6
:10292000F70180810E94A21C0F5F1F4F0894E11CD9
:10293000F11CF2E00E3C1F07E1F683E08093C40235
:102940000E94F80481E080937A035D980E94A71B9F
:102950005B016C010E94991B2B013C018091740367
:10296000823008F065C0E0903403F09035030091A8
:102970003603109137038091380390913903A09169
:102980003A03B0913B038E159F05A007B10709F4E8
:102990004FC080EE92E00E943801A60195012E19E9
:1029A0003F09400B510B6C5D7540804090406217B1
:1029B000730784079507E0F5E0923803F092390336
:1029C00000933A0310933B030E943F038093470315
:1029D0002091450330914603280F311D3093460363
:1029E00020934503609144036F5F60934403693013
:1029F000F8F0C90170E00E94FA20CB017093460301
:102A0000609345032091480343E0249F90011124E3
:102A1000820F931F96958795969587958093480387
:102A20000E94A10D10924603109245031092440398
:102A3000809173039090F103882309F463C180901F
:102A40007403891408F0E1C180EE92E00E9438011D
:102A50002091340330913503409136035091370370
:102A6000A21AB30AC40AD50A68517C4F8F4F9F4FF0
:102A70006A157B058C059D0508F077C080914C0395
:102A800090914D03880F991F90934D0380934C03B1
:102A900081E080937A03882081F440923C03509235
:102AA0003D0360923E0370923F03109240031092E8
:102AB00041031092420310924303809174038F5F8D
:102AC0008093740380EE92E00E94380120913403D9
:102AD000309135034091360350913703260F371F4D
:102AE000481F591F20933403309335034093360316
:102AF0005093370381E080937A035E9A0E94860D9B
:102B00000E94A10D32C080EE92E00E9438019B012C
:102B1000AC018091340390913503A0913603B091BC
:102B2000370386017501E81AF90A0A0B1B0B682D99
:102B300070E080E090E00E94DB206E157F0580074A
:102B4000910798F410924D0310924C0381E080930A
:102B50007A03109248030E94A10DA0923403B09210
:102B60003503C0923603D0923703809174038823D3
:102B700009F4F2C09091DD02992389F1809152030A
:102B8000882369F5892F90E00E94E50020913C039D
:102B900030913D0340913E0350913F038301720108
:102BA000E21AF30A040B150B6E157F0580079107D7
:102BB000B0F481E0809352030E94E2078091D90231
:102BC0000E941801640D751D861D971D616060933C
:102BD0004003709341038093420390934303909189
:102BE000DF029923F1F0809150038823D1F4892FDB
:102BF00090E00E94E50020913C0330913D0340911C
:102C00003E0350913F0383017201E21AF30A040B61
:102C1000150B6E157F058007910718F481E08093EE
:102C200050039091DE029923F1F0809151038823A3
:102C3000D1F4892F90E00E94E50020913C0330916F
:102C40003D0340913E0350913F0383017201E21A1C
:102C5000F30A040B150B6E157F058007910718F416
:102C600081E0809351038091D5029091D602A0918A
:102C7000D702B091D8020097A105B10509F46CC044
:102C80008091400390914103A0914203B09143038E
:102C90000097A105B10509F45FC083017201E81A2C
:102CA000F90A0A0B1B0B17FD57C06091DA0270E09E
:102CB00080E090E028EE33E040E050E00E94DB202E
:102CC0006E157F058007910708F046C08091D302FA
:102CD00090E0E4E096958795EA95E1F781700E948F
:102CE000191280E00E9419040E94F8040E94991BA6
:102CF000616060934003709341038093420390931B
:102D000043032AC080EE92E00E9438019B01AC018F
:102D10008091340390913503A0913603B09137032D
:102D200086017501E81AF90A0A0B1B0B692D70E080
:102D300080E090E00E94DB206E157F058007910700
:102D400058F4A0923403B0923503C0923603D09267
:102D5000370381E080937A03809151038823B1F493
:102D60008091CD02883219F40E94AC0A0FC08932DA
:102D700039F480915203609174030E94890B06C05C
:102D80008A3221F4809152030E94200B80917A03B1
:102D90008823B9F0E0913303EF5FE0933303E83128
:102DA00031F0F0E0E052FD4F8785882311F4109256
:102DB0003303809133030E9429030E94480A109232
:102DC0007A03809175038F3F21F50E94991B209112
:102DD0007603309177034091780350917903621B19
:102DE000730B840B950B695E73408040904088F0B4
:102DF0000E94991B60937603709377038093780306
:102E0000909379030E94710A04C0891409F0ADCE31
:102E10007ACE6696E0E10C946921FF920F931F939E
:102E2000082FF62E61E00E94361C802F61E00E9480
:102E3000A21C8F2D61E00E94A21C8AE090E00E94FB
:102E4000F11B8F2D0E94D51C892B11F410E00FC0AF
:102E5000802F60E00E94A21C8AE090E00E94F11B9B
:102E60008F2D0E94D51C10E0892B09F411E0802FD2
:102E700060E00E94361C802F60E00E94A21C8F2D13
:102E800060E00E94A21C812F1F910F91FF90089576
:102E9000EF92FF920F931F937C010CE814E0C8019E
:102EA0006F2D70E04AE050E00E940C1EC8016EE2F7
:102EB0000E944B1DB701E4E076956795EA95E1F72E
:102EC0006F707070C8014AE050E00E940C1EC8018B
:102ED0006EE20E944B1D8FE0E822FF24C801B7017B
:102EE0004AE050E00E940C1E1F910F91FF90EF905E
:102EF0000895A2E2B0E0EFE7F7E10C944B218E01D8
:102F00000F5F1F4F80E1D8011D928A95E9F78CE889
:102F100094E066E371E00E948F1E0E943C0F20E463
:102F200031EE4DE958E12F8F38A349A35AA380EC25
:102F300091EDA8E9BBE18B8F9C8FAD8FBE8F24EF05
:102F400031E040E050E02F8B388F498F5A8F80E579
:102F5000C82E83ECD82EE12CF12CB0E44B2EB1EE30
:102F60005B2EBDE96B2EB8E17B2E88249924540199
:102F700033241E8A1D8A198A1A8A1B8A1C8AFFC05A
:102F80008CE894E00E940E208434B9F0853430F44B
:102F90008332B9F18C3209F0CCC044C0833509F0DA
:102FA000C8C02F8D38A149A15AA1C901DA012C014D
:102FB0003D01882499245401E2C08CE894E064E443
:102FC0000E944B1D8CE894E040E451EE6DE978E1FD
:102FD0002AE030E00E942F1E8CE894E06CE20E9410
:102FE0004B1D8CE894E040EC51ED68E97BE12AE070
:102FF00030E00E942F1E8CE894E06CE20E94691D74
:10300000BEC019821A821B821C821D821E821F82F0
:10301000188619861A861B861C861D861E861F86A4
:10302000188A3AC0339434E0331609F0A8C0698195
:103030007A818B819C8128EE33E040E050E00E9451
:10304000DB206F8F78A389A39AA36D817E818F8106
:1030500098850E94DB206B8F7C8F8D8F9E8F89855A
:103060009A85AB85BC858F8B988FA98FBA8F6D851C
:103070007E858F8598890E94DB206B017C0190E220
:10308000C9169EE4D90690E0E90690E0F90630F40E
:103090008CE162E30E941E03332471C0A0E3CA16D0
:1030A000A5E7DA06A0E0EA06A0E0FA0618F48CE14B
:1030B00062E2F0CFB0E4CB16BCE9DB06B0E0EB0691
:1030C000B0E0FB0618F48CE166E2E4CFE0E5CE1652
:1030D000E3ECDE06E0E0EE06E0E0FE0618F48CE14C
:1030E00062E1D8CFF0E6CF16FAEEDF06F0E0EF06A9
:1030F000F0E0FF0618F48CE165E1CCCF20E7C216C2
:1031000021E1D20621E0E20620E0F20618F48CE18B
:1031100061E0C0CF30EAC31636E8D30631E0E306FB
:1031200030E0F30618F48CE163E0B4CF8CE165E0A5
:10313000B1CFA0ED2A2E280E49E0421500F1032D53
:1031400010E0000F111F000F111F81E090E08C0FA5
:103150009D1F080F191FD8016D917D918D919C9134
:103160002AE030E040E050E00E94DB20620D711D5B
:10317000811D911DF80160837183828393838CE8A4
:1031800094E00E94D41F892B09F0FACE8114910497
:10319000A104B10489F4C301B2010E94AF0361E04C
:1031A00070E080E090E00E94CD1BFFEFFE8B1D8A57
:1031B000198A1A8A1B8A1C8A2F89388D498D5A8D43
:1031C00082169306A406B506E0F40E943F032989FF
:1031D0003A894B895C89280F311D411D511D298B6E
:1031E0003A8B4B8B5C8B3D89381708F48D8B4E895D
:1031F000841708F48E8B0894811C911CA11CB11CAF
:1032000056C0C301B20128EE33E040E050E00E9416
:103210000E218CE894E0BA01A9012AE030E00E9476
:10322000FD1D8CE894E06CE20E944B1D8CE894E05C
:103230006D894AE050E00E941D1E8CE894E06CE22B
:103240000E944B1D69897A898B899C89A50194010B
:103250000E940E218CE894E0BA01A9012AE030E036
:103260000E94FD1D8CE894E06CE20E944B1D8CE8EE
:1032700094E06E894AE050E00E941D1E8CE894E0C4
:103280006CE20E94691D4C0C5D1C6E1C7F1C8B8DBA
:103290009C8DAD8DBE8D84159505A605B70520F4D2
:1032A0004F8C58A069A07AA08824992454012F8DAE
:1032B00038A149A15AA1285E33404040504009F04E
:1032C0005ECFA296E2E10C94672180E065E970E0B0
:1032D00042E050E00E94D41A0895A1E0B0E0E3E794
:1032E000F9E10C945B2180E00E94B10085E061E08F
:1032F0000E94361C86E061E00E94361C0E94270F67
:1033000080E060E00E94361C81E061E00E94361C93
:103310008CE894E040E052EC61E070E00E944D1FC8
:103320000E94BB110E9430108CE894E063E471E0CD
:103330000E948C1E83E793E00E9448178CE894E07B
:103340006AE571E00E948C1E8CE894E067E070E012
:103350004AE050E00E94781E0E94651978945E9AB7
:1033600083E063E10E940D17882329F05E985D9841
:103370000E947917FBCF89E062E10E940D17882334
:1033800029F40E94CA11882309F006C18CE894E050
:1033900062E671E00E948C1E60E070E080E090E0E8
:1033A0000E948910882349F00E94C5118CE894E09E
:1033B0006BE971E00E948F1E5D9A0E94210E22C06F
:1033C0008091C902833229F08091D3028B7F809350
:1033D000D3028091D30281FF15C082FD13C064EF38
:1033E00071E080E090E00E948910882359F00E94EB
:1033F000C5118CE894E06BE971E00E948F1E0E9479
:10340000210E5D9A8091C702823239F58091C902FE
:10341000833219F581E00E94DA0D8091D30282FF98
:1034200009C08CE894E066EB71E00E948F1E0E9458
:103430006F0813C064E170E080E090E00E94CD1B53
:1034400080E2BE016F5F7F4F41E021E00E94EC0807
:10345000882319F481E0809375038CE894E061EC93
:1034600071E00E948C1E8FE00E94B10080E00E94FB
:1034700019041092330380E00E9429031092F10393
:1034800090E0983158F4292F2F5FE92FF0E0E052B7
:10349000FD4F8785882311F0922FF3CF9093F1038E
:1034A00083E08093C4020E943C0F809175038823BF
:1034B00011F00E94710A8091CD02883211F08A3297
:1034C00039F48CE894E040E052EC61E070E02BC00D
:1034D000893271F48CE894E040EA56E861E070E0EB
:1034E0000E944D1F8091C20080628093C20022C062
:1034F000809108038871803169F04091E102509118
:10350000E2026091E3027091E4024A3051056105E4
:10351000710538F48CE894E040E855E260E070E032
:1035200002C08CE894E00E944D1F04C08CE894E037
:103530000E940E208CE894E00E94D41F892BB1F7E2
:103540008091CC02843229F08091C1008F7E8093DB
:10355000C1008091CD02853259F08A3249F089321A
:1035600039F0883229F08091C100877F8093C100B3
:103570001092EF031092F003109273030E94A71BA6
:10358000609334037093350380933603909337032D
:103590002196E2E00C9477210E94210E8091C702CF
:1035A000823209F011CF0CCF823000F5E82FF0E025
:1035B000EE0FFF1FE950FC4F71836083882319F0E1
:1035C0008130A1F408C0809169008C7F842B8093A6
:1035D0006900E89A089580916900440F551F440FCF
:1035E000551F837F842B80936900E99A08951F9269
:1035F0000F920FB60F9211242F933F934F935F9327
:103600006F937F938F939F93AF93BF93EF93FF93AA
:103610008091F7039091F803892B29F0E091F7034B
:10362000F091F8030995FF91EF91BF91AF919F91B0
:103630008F917F916F915F914F913F912F910F905B
:103640000FBE0F901F9018951F920F920FB60F92FA
:1036500011242F933F934F935F936F937F938F9397
:103660009F93AF93BF93EF93FF938091F903909152
:10367000FA03892B29F0E091F903F091FA030995F7
:10368000FF91EF91BF91AF919F918F917F916F913A
:103690005F914F913F912F910F900FBE0F901F9010
:1036A00018951F920F920FB60F9211242F933F93EC
:1036B0008F939F93AF93BF938091FF0390910004EA
:1036C000A0910104B0910204309103040196A11D60
:1036D000B11D232F2D5F2D3720F02D570196A11DF1
:1036E000B11D209303048093FF0390930004A093E3
:1036F0000104B09302048091FB039091FC03A0911C
:10370000FD03B091FE030196A11DB11D8093FB0343
:103710009093FC03A093FD03B093FE03BF91AF9180
:103720009F918F913F912F910F900FBE0F901F90FF
:1037300018958FB7F8942091FF03309100044091C1
:103740000104509102048FBFB901CA0108959FB7C7
:10375000F8942091FB033091FC034091FD035091BC
:10376000FE0386B5A89B06C08F3F21F02F5F3F4F19
:103770004F4F5F4F9FBF542F432F322F2227280FC9
:10378000311D411D511D82E0220F331F441F551F63
:103790008A95D1F7B901CA010895EF92FF920F936C
:1037A0001F93CF93DF937B018C010E94A71BEB013A
:1037B0000EC00E94A71B6C1B7D0B685E7340C8F394
:1037C0000894E108F10801091109C851DC4FE1141E
:1037D000F1040105110569F7CDB7DEB7E6E00C94F9
:1037E0007321019739F0880F991F880F991F02974D
:1037F0000197F1F70895789484B5826084BD84B50B
:10380000816084BD85B5826085BD85B5816085BDDB
:10381000EEE6F0E0808181608083E1E8F0E01082F4
:10382000808182608083808181608083E0E8F0E035
:10383000808181608083E1EBF0E08081846080831F
:10384000E0EBF0E0808181608083EAE7F0E0808156
:1038500084608083808182608083808181608083B6
:103860008081806880831092C1000895CF93DF9398
:10387000482F50E0CA0186569F4FFC0134914A57A9
:103880005F4FFA018491882369F190E0880F991FB6
:10389000FC01E859FF4FA591B491FC01EE58FF4F90
:1038A000C591D491662351F42FB7F8948C91932F3E
:1038B000909589238C93888189230BC0623061F4B1
:1038C0002FB7F8948C91932F909589238C938881AE
:1038D000832B88832FBF06C09FB7F8948C91832BCE
:1038E0008C939FBFDF91CF910895833071F0843026
:1038F00028F48130A1F0823021F514C08630B1F077
:103900008730D1F08430E9F404C0809180008F7753
:1039100003C0809180008F7D80938000089584B5DE
:103920008F7702C084B58F7D84BD08958091B000EB
:103930008F778093B00008958091B0008F7D809341
:10394000B0000895FF920F931F93F62E482F50E07A
:10395000CA0182559F4FFC012491CA0186569F4F90
:10396000FC0114914A575F4FFA0104910023C9F0FA
:10397000222319F0822F0E94751CE02FF0E0EE0F39
:10398000FF1FEE58FF4FA591B4919FB7F894FF2009
:1039900021F48C911095812302C08C91812B8C9302
:1039A0009FBF1F910F91FF9008950F931F93482F72
:1039B00050E0CA0182559F4FFC012491CA018656EE
:1039C0009F4FFC0104914A575F4FFA011491112354
:1039D00019F420E030E015C0222319F0822F0E9454
:1039E000751C812F90E0880F991F84589F4FFC0110
:1039F000A591B4918C9120E030E0802311F021E07A
:103A000030E0C9011F910F910895982F8E3008F072
:103A10009E50977080918B028295880F880F807CD2
:103A2000892B80937C0080917A00806480937A0057
:103A300080917A0086FDFCCF20917800409179003A
:103A4000942F80E030E0282B392BC9010895A0E0A5
:103A5000B0E0EDE2FDE10C9455217C016B018A019F
:103A6000C0E0D0E00FC0D6016D916D01D701ED919E
:103A7000FC910190F081E02DC7010995C80FD91F75
:103A8000015010400115110571F7CE01CDB7DEB719
:103A9000E8E00C947121DC01ED91FC910190F08142
:103AA000E02D09950895EF92FF920F931F938C01DB
:103AB0006DE00E944B1D7C01C8016AE00E944B1D15
:103AC0009C012E0D3F1DC9011F910F91FF90EF909A
:103AD0000895EF92FF920F931F937C010E944B1D5C
:103AE0008C01C7010E94531D9C01200F311FC90189
:103AF0001F910F91FF90EF900895CF93DF93EC010A
:103B00006115710519F420E030E00FC0DB010D9064
:103B10000020E9F71197A61BB70BE881F981028015
:103B2000F381E02DAD0109959C01C901DF91CF9191
:103B300008954F925F927F928F929F92AF92BF9221
:103B4000CF92DF92EF92FF920F931F93DF93CF9369
:103B5000CDB7DEB7A1970FB6F894DEBF0FBECDBFCD
:103B60002C01742ECB01223008F42AE019A231E294
:103B7000C32ED12CCC0EDD1E822E9924AA24BB2468
:103B8000672D752FA50194010E940E2179018A01EC
:103B9000C801B701A50194010E94DB20472D461BF7
:103BA0000894C108D1084A3010F4405D01C0495C56
:103BB000F6014083E114F1040105110521F07E2C8A
:103BC0005F2DC801DDCFC201B6010E947D1DA19607
:103BD0000FB6F894DEBF0FBECDBFCF91DF911F911E
:103BE0000F91FF90EF90DF90CF90BF90AF909F909C
:103BF0008F907F905F904F900895DC0121153105E3
:103C000041F4ED91FC910190F081E02D642F099534
:103C100008950E94991D0895EF92FF920F931F93AC
:103C20009A017B0100E010E0B801A7010E94FD1D90
:103C30001F910F91FF90EF900895EF92FF920F93D5
:103C40001F939A01E62EFF2400E010E0B801A701BF
:103C50000E94FD1D1F910F91FF90EF900895A0E02D
:103C6000B0E0E5E3FEE10C945521EC016A017B0133
:103C70002115310541F4E881F9810190F081E02DB1
:103C8000642F09951BC02A303105B1F477FF13C0AA
:103C90006DE20E944B1D8C0144275527BA014C1937
:103CA0005D096E097F09CE012AE00E94991D9C01E1
:103CB000200F311F04C02AE00E94991D9C01C901F8
:103CC000CDB7DEB7E8E00C947121EF92FF920F932D
:103CD0001F937B019A010027F7FC0095102FB80174
:103CE000A7010E942F1E1F910F91FF90EF90089542
:103CF000EF92FF920F931F937C010E94651E8C012F
:103D0000C7010E94531D9C01200F311FC9011F9143
:103D10000F91FF90EF9008950E947D1D0895EF92FE
:103D2000FF920F931F937C010E948C1E8C01C70190
:103D30000E94531D9C01200F311FC9011F910F913B
:103D4000FF90EF90089508951F920F920FB60F9273
:103D500011242F933F934F938F939F93EF93FF9350
:103D60008091C00082FD1DC04091C6002091440496
:103D7000309145042F5F3F4F2F7330708091460480
:103D8000909147042817390771F0E0914404F091AD
:103D90004504EC5FFB4F408330934504209344047B
:103DA00002C08091C600FF91EF919F918F914F913A
:103DB0003F912F910F900FBE0F901F9018951F925B
:103DC0000F920FB60F9211242F933F938F939F93CF
:103DD000EF93FF93209188043091890480918A04A5
:103DE00090918B042817390731F48091C1008F7DA1
:103DF0008093C10014C0E0918A04F0918B04E85BC9
:103E0000FB4F208180918A0490918B0401968F73DF
:103E1000907090938B0480938A042093C600FF9146
:103E2000EF919F918F913F912F910F900FBE0F9027
:103E30001F901895A0E0B0E0E0E2FFE10C94512162
:103E4000FC011382128288EE93E0A0E0B0E084834C
:103E50009583A683B78388EB92E0918380837587EF
:103E6000648757874687318B208B138B028BF58AAB
:103E7000E48AD78AC68AB18EA08E938E828E8F8571
:103E8000848F8889858F8989868F8A89878F8B8996
:103E900080A32096ECE00C946D21AF92BF92DF924C
:103EA000EF92FF920F931F93CF93DF93EC017A0170
:103EB0008B01DD24403081EE580780E0680780E008
:103EC000780711F0DD24D39491E0A92EB12CEC8970
:103ED000FD89DD2069F0C50108A002C0880F991F87
:103EE0000A94E2F7808360E079E08DE390E005C01A
:103EF000108260E874E88EE190E0A80197010E94CA
:103F00000E212150304040405040569547953795FE
:103F1000279580E12030380720F0DD2011F0DD24E6
:103F2000D6CFE889F9893083EA89FB89208319A2F1
:103F3000EE89FF89408121E030E0C9010C8C02C08C
:103F4000880F991F0A94E2F7482B4083EE89FF8976
:103F50004081C9010D8C02C0880F991F0A94E2F7B5
:103F6000482B4083EE89FF894081C9010E8C02C035
:103F7000880F991F0A94E2F7482B4083EE89FF8946
:103F800080810F8C02C0220F331F0A94E2F7209524
:103F900028232083DF91CF911F910F91FF90EF9005
:103FA000DF90BF90AF900895DC011C96ED91FC91DD
:103FB0001D97E05CFF4F2191319180819181281BF9
:103FC000390B2F733070C90108958CE894E00E947A
:103FD000D41F892B11F00E94A31E0895DC011C96AA
:103FE000ED91FC911D97E05CFF4F20813181E05401
:103FF000F040DF01AE5BBF4F8D919C911197281768
:10400000390719F42FEF3FEF07C08D919C91E80F0E
:10401000F91F8081282F30E0C9010895DC011C962A
:10402000ED91FC911D97E05CFF4F20813181E054C0
:10403000F040DF01AE5BBF4F8D919C911197281727
:10404000390719F42FEF3FEF10C08D919C91119714
:10405000E80FF91F20818D919C91119701968F7324
:10406000907011969C938E9330E0C9010895DC0105
:1040700091968C919197882339F05496ED91FC910B
:104080005597808186FFF9CF91961C920895CF9322
:10409000DF93EC01EE85FF85E05CFF4F20813181ED
:1040A000E054F0402F5F3F4F2F733070DF01AE5B65
:1040B000BF4F8D919C91119728173907D1F3E05C80
:1040C000FF4F80819181E054F040E80FF91F608339
:1040D000EE85FF85E05CFF4F31832083EE89FF8909
:1040E000208181E090E00F8C02C0880F991F0A9414
:1040F000E2F7282B208381E089A3EC89FD89808168
:104100008064808381E090E0DF91CF9108958F9269
:104110009F92AF92BF92CF92DF92EF92FF920F9356
:104120001F9300D000D00F92EDB7FEB7319684E018
:10413000ADB7BEB711968C9383E0818387E082830D
:1041400085E0838381E084838CE894E064E074E01C
:1041500048E454E025EC30E004EC10E0B0ECEB2E49
:10416000F12CA1ECCA2ED12CF2ECAF2EB12CE6EC46
:104170008E2E912C0E941A1F0F900F900F900F906F
:104180000F901F910F91FF90EF90DF90CF90BF9015
:10419000AF909F908F900895CF93DF930E94FB1B69
:1041A0000E946D19C5EEDFE10E94E5122097E1F350
:1041B0000E94E51FF9CF629FD001739FF001829F9B
:1041C000E00DF11D649FE00DF11D929FF00D839FA6
:1041D000F00D749FF00D659FF00D9927729FB00D43
:1041E000E11DF91F639FB00DE11DF91FBD01CF0156
:1041F00011240895AA1BBB1B51E107C0AA1FBB1FB6
:10420000A617B70710F0A61BB70B881F991F5A9562
:10421000A9F780959095BC01CD010895A1E21A2ED1
:10422000AA1BBB1BFD010DC0AA1FBB1FEE1FFF1F5A
:10423000A217B307E407F50720F0A21BB30BE40BAA
:10424000F50B661F771F881F991F1A9469F76095F1
:104250007095809590959B01AC01BD01CF010895AB
:1042600097FB092E05260ED057FD04D0D7DF0AD0C4
:10427000001C38F450954095309521953F4F4F4F95
:104280005F4F0895F6F790958095709561957F4FF3
:104290008F4F9F4F08952F923F924F925F926F9250
:1042A0007F928F929F92AF92BF92CF92DF92EF92C6
:1042B000FF920F931F93CF93DF93CDB7DEB7CA1B47
:1042C000DB0B0FB6F894DEBF0FBECDBF09942A8872
:1042D000398848885F846E847D848C849B84AA841A
:1042E000B984C884DF80EE80FD800C811B81AA81A7
:1042F000B981CE0FD11D0FB6F894DEBF0FBECDBF72
:10430000ED010895EE0FFF1F0590F491E02D099443
:04431000F894FFCF4F
:1043140054582074696D656F757421005761697410
:10432400696E672062696E640A00476F7420706B5F
:10433400740A006461746120676F6F640A005258E4
:104344002068616E67007363616E6E6572206D6FC5
:104354006465004F70656E4C52536E67205258204E
:104364007374617274696E672000206F6E20485701
:104374002000454550524F4D2064617461206E6F9A
:10438400742076616C6964206F722062696E6420A7
:104394006A756D70706572207365742C20666F7217
:1043A40063696E672062696E640A005361766564AE
:1043B4002062696E64206461746120746F204545D5
:1043C40050524F4D0A004920616D20736C6176652F
:1043D40000456E746572696E67206E6F726D616CF4
:1043E400206D6F646500002001220126022102274E
:1043F4000323032604260526052B06240725072860
:104404000729072AC01200001A400AA1204EA5005D
:104414001B1E27522C23308025000005400AA120B2
:104424004EA50020244EA52C2330004B000006404E
:104434000AD0009D49007B289D492C233000E100CF
:104444000005400A4501D7DC03B81E0EBF00232E29
:1044540048E801008A400A6001555502AD1E20005B
:104464000023C88025000005400AA1204EA5002095
:10447400244EA52C23300002000200020002000298
:104484000002000200020002000200020002000218
:104494000002000200028813409C08010912031361
:1044A4000E0F0001020000001000000008002000B0
:1044B40000010000020000000100000200070B0CD4
:1044C40010111500000000004720271DD41F0E20E6
:0444D400EE1F372080
:107E00000F92CDB7DEB7112484B714BE81FFF1D035
:107E100082E08093C00088E18093C10086E0809377
:107E2000C20080E18093C4008EE0CDD088249924E4
:107E3000CC24C394F5E0DF2EE1E1EE2E73E0F72EC3
:107E4000B6D0082F813479F4B2D08983C2D0898129
:107E5000823811F481E005C0813811F485E001C059
:107E600083E09ED09AC0823411F484E103C085344B
:107E700019F485E0B6D091C0853561F498D0082F0B
:107E800010E095D090E0982E8824802A912A880CC2
:107E9000991C82C0863521F484E0A3D080E0E1CF34
:107EA000843609F04CC083D082D0A82E80D0B82E62
:107EB00000E011E07CD0F80181938F01AE16D1F77C
:107EC00088D0FB2DF53489F4E0E0F1E00BC0F9999E
:107ED000FECF92BC81BC0894811C911C819180BD15
:107EE000FA9AF99AEA1598F358C08B2D863409F05E
:107EF00054C0F401F7BEE89507B600FCFDCFF401CD
:107F0000A0E0B1E02C9130E011968C91119790E0B7
:107F1000982F8827822B932B12960C01C7BEE895C9
:107F20001124329681E0A038B80761F7F401D7BE7A
:107F3000E89507B600FCFDCFE7BEE8952EC0843774
:107F4000F1F435D034D0182F32D0B82E42D0FB2DDA
:107F5000F63421F4F40105914F010CC0FB2DF534EA
:107F600049F4F999FECF92BC81BC0894811C911C04
:107F7000F89A00B5802F14D0115049F70EC08537FC
:107F800039F427D08EE10CD085E90AD08FE069CF93
:107F9000813511F488E017D01CD080E101D050CF9A
:107FA0009091C00095FFFCCF8093C600089580910A
:107FB000C00087FFFCCF8091C00084FD01C0A89560
:107FC0008091C6000895E0E6F0E098E19083808318
:107FD0000895EDDF803219F088E0F5DFFFCF84E10E
:107FE000DFCF1F93182FE3DF1150E9F7F2DF1F9166
:0E7FF0000895282E80E0E7DFEE27FF27099492
:027FFE0001057B
:0400000300007E007B
:00000001FF
